:030000000219FDE5
:03000B000200A848
:03002B0002015A75
:03005B000202EBB3
:030073000202D8AE
:1000800002030406080C10182030406080040608A3
:100090000C10182030406080A0C00003070F1F051F
:1000A000050D050305030302C2AFC0D0C0E0206206
:1000B00014E5256009E473E525F4F58AD262D0E001
:1000C000D0D0D2AF3285268AC262E526F4602F30C6
:1000D000682520720DD0E0D0D0C295C293C297D2CD
:1000E000AF32C295C293C297206F0C206509740984
:1000F000D5E0FDE57B4290D0E0D0D0D2AF32758A1A
:1001000000C28DD26201F701B7306805206502D2C6
:100110009501B7306805206502D29701B7306805B0
:10012000206502D29301B7C29430680A2065077433
:1001300009D5E0FDD29501B7C29630680A2065075F
:100140007409D5E0FDD29701B7C29230680A2065E4
:10015000077409D5E0FDD29301B7C2AFC2AD53E633
:10016000EFC0D0C0E0D2D3D2AFC2CEE52A60072024
:10017000744F152A21C17800790020742EE5803053
:100180007E01F430E50278FF53DACF207E0343DAB4
:1001900020307E0343DA10C2D8C271E580307E0180
:1001A000F430E50279FFC3E89970CB306103752A1A
:1001B00018207403752A18885CD270E86003755F94
:1001C0000020740DE52B6004152B21D143DA01C208
:1001D000D82070024144A85C206102C270207431B2
:1001E000C3E894F0400374F0F8E8C4540F28F87999
:1001F00084B703024111C313C3138721200802C32C
:1002000013200A06C3C898F8411128F8500374FF58
:10021000F8C3E895655003E565F88822E52D540696
:100220006022206B1FE536C333C333F8E564C31384
:10023000C313F9C3952240028922E82522F52250F2
:10024000037522FF852224A824C3E524956140027A
:10025000A8618825E56670024188C3E8AA669A50BD
:1002600003E8FAE4F9EAC333FBE568F45B29400DDF
:100270002567F8E56760021567400B41880AC3E50A
:10028000679A5002056778FF8826C26FC3E52694F7
:10029000F84002D26F20CF0AD0E0D0D043E610D28F
:1002A000AD32C2CF053A7801E52A600530740215F7
:1002B0002AC3E55C94014005755F0041CE7560007E
:1002C000756900E55F2401F55F5003755FFFD0E0BD
:1002D000D0D043E610D2AD32C2AF53E67F7592FA6A
:1002E0007593FFC260759104D2AF32C2AF53E6EF8F
:1002F000C2ADC0D0C0E0C0F0D2D3D2AFA8FBA9FC41
:10030000C2D8307102615253DACF207E0343DA1033
:10031000307E0343DA20D271E580307E01F420E59F
:1003200002612988278928A17F53DACF207E0343E1
:10033000DA20307E0343DA10C2D8C271307402A1D1
:100340006B7800E580307E01F430E502A16B885CBB
:10035000A15353DACF207E0343DA20307E0343DA01
:1003600010C271206102812B53DACF207E0343DA61
:1003700010307E0343DA20C2D8D27188578958C31F
:10038000E89555F8E99556F97B007E087A00C3E8B0
:10039000948CE994005005755B00811D882178A23A
:1003A000E6A8216055C3E894C8E994005008E4D257
:1003B000E4FB7A0A61F8C3E89468E994015008E420
:1003C000D2E3FB7A0F61F8C3E894D0E994025008B5
:1003D000E4D2E2FB7A1E61F8C3E894A0E9940550E8
:1003E00008E4D2E1FB7A3C61F8C3E89498E9940808
:1003F0005008E4D2E0FB7A787E00C3E89559FCE926
:10040000955AFD30E70AECF42401FCEDF43400FDCC
:10041000755B00C3EC9AED9E5003755B01885989AA
:100420005A8557558558567802A153C3E89527F841
:10043000E99528F9307C02A137307B02A137307A68
:1004400002A130207502814EE9FDE8FC816DE9C30F
:1004500013F9E813F8307902A130E9C313F9E8136E
:10046000F8307802A130E9C313FDE813FC20612CB9
:0F047000C3EC941CED940240028184ED701EC316
:10047F00EC94C850180529E52970021529C3E52900
:10048F00940A5002A16B755C00D270A16BE52960D4
:10049F000215297888E6F97400207F087896B90349
:1004AF0002789EE624FAFEE43400FFC3EC9EFCEDD6
:1004BF009FFD9208B90310A2085007207609D27643
:1004CF0081D6307602C276A2085016B9030DECF42D
:1004DF002401FCEDF43400FD0204F078007900A152
:1004EF0037B90315EC33FCED33FDC3EC940AFCED87
:1004FF009400FD50047C007D00C3EC94FFED94004C
:10050F00400678FF7900A137EC8572F0A4C5F0A200
:10051F00F733F87900400302055378FF790002059D
:10052F0053E9C313F9E813F8307C0EE9600278FF42
:10053F00C3E81338F8E43400F9C3E894FFE99400F2
:10054F00400278FF885CD270206102A16B741FF4A7
:10055F00552F4BF52FC274EB7002D274752A1830D9
:10056F007403752A0A306102A17F20740353DAFEE7
:10057F00207403752B06D0F0D0E0D0D0D2AD43E677
:10058F00103279010205AF79030205AF790A02052E
:10059F00AF791E0205AF79640205AF79C80205AFC6
:1005AF007817E4D5E0FDD8FAD9F6227A147B7802D1
:1005BF0005D67A107B8C0205D67A0D7BB40205D650
:1005CF007A0B7BC80205D6E573D5E001227902E4E8
:1005DF00C296D5E0FDD297D5E0FDC297D5E0FDD20A
:1005EF0096D5E0FDE920E002D29530E002D293E506
:1005FF0073D5E0FDE920E002C29530E002C29374AA
:10060F0096D5E0FDD9C9EAF8D5E0FDD8FBDBB8C235
:10061F009622C37C007D0075F00005F0EA33FAEBFB
:10062F0033FB50F6EB13FBEA13FAC3E9FFE8FEE8DE
:10063F009AF8E99BF95004EFF9EEF8B3EC33FCEDBF
:10064F0033FDD5F0DFEDF9ECF822E889F08A20D2FE
:10065F00D4F8A9F07B0030F70B7BFFF42401F8E905
:10066F00F43400F9E88520F0A4ADF0F8E98520F026
:10067F00A4AFF0FEED2EF974003FFA7C04C3EA1329
:10068F00FAE913F9E813F8DCF48BF030F70AE8F421
:10069F002401F8E9F43400F9E889F0C2D4F8A9F09C
:1006AF002222C3E54113F9E54013F8C3E54498F856
:1006BF00E54599F9500CC3E89480E994FF40160280
:1006CF0006E8C3E8947FE9940050030206E8787FB8
:1006DF0079000206E8788079FF8849894A22E5493E
:1006EF002546F8E54A3547F9854A20E4300701F4F5
:1006FF003548FA30E709C3EA94F04015020726C3DC
:10070F00EA940F500302072678FF79FF7A0F02074A
:10071F0026780079007AF0C3E5249561500AC374F6
:10072F00019524500B020744E54A20E70E020744C7
:10073F00E54A30E706884689478A482278A5E6FACF
:10074F00C3E54933F8E54A33F9D159E930E70BC32B
:10075F00E89480E994FF4013E17EC3E8947FE99425
:10076F00005002E17E787F7900E17E788079FFE8A2
:10077F0020E715C3E52398F84009C3E89401400327
:10078F000207A578010207A5E8F424012523F84004
:10079F00030207A578FF884B2278A6E6FAA847A997
:1007AF0048D159E930E70CC3E89401E994FF4016AA
:1007BF000207D9C3E894FFE9940050030207D978E0
:1007CF00FF79000207D9780179FFE920E715C3E522
:1007DF004B98F84009C3E8940140030208007801E0
:1007EF00020800E8F42401254BF8400302080078C2
:1007FF00FF88242278FF20692879A1E76023E5414B
:10080F00601F74FF8541F0848539F0306A0375F0FD
:10081F0005A4F8C5F0600278FFC3E895645002A8FC
:10082F0064886322C3E5409440E5419401E5635039
:10083F0003140144046002F5632202084C2275E898
:10084F0090227883E6FF30EDF9A8BDA9BE0570C3ED
:10085F00E57094084052757000E9FA79A0E760449A
:0E086F00EA7007E571601B020885C3E8957109
:10087D006010E5715006600C140208910460F902D5
:10088D000891E571F571C3946D401B7561C0C394FA
:10089D00044013756180C39404400B756140C3948B
:1008AD0004400375610075BB0822E561F460020523
:1008BD0061E570B4070375BB1022743279A787F018
:1008CD00A4C5F0A2F733F8C3E895614002A861888A
:1008DD00228824882588268864227540007541F079
:1008ED0022C2AF75C820A8CCA9CDAA3A30CF010A33
:1008FD0075C824D2AFAB3BAC3C883B893CC3E89B6D
:10090D00F8E99C206908F930660221FF2159AD3DB7
:10091D008A3DF9EA9DFA600678FF79FF213EAE3EE9
:10092D00AF3F8B3E8C3FA83BA93CC3E89EF8E99FA7
:10093D00F9C3E54113FBE54013FAE82AF540E93B1D
:10094D00F54150067540FF7541FF21A6AA40AB4108
:10095D00AC40AD417E047F02C3EB9404400D1E1FDD
:10096D00C3EB94084005206A021E1FC3ED13FDEC76
:10097D0013FCDEF7C3EA9CFAEB9DFBEF6009C3E9BC
:10098D0013F9E813F8DFF7EA28FAEB39FB8A408B05
:10099D004150067BFF8B408B41C3EB94025002D23A
:1009AD00663069047F0321D17892E6FFC3E5379461
:1009BD008240110FC3E53794A040010FC3EF940699
:1009CD0040027F057E02E541C4540FF9E541C45450
:1009DD00F0F8E540C4540F28F8C3E89EFAE99400F6
:1009ED00FB4009C3EA9402EB940050047A02E4FB45
:1009FD00414BAA40AB41EBC4FEEAC4540F4EFCC3BD
:100A0D00EA9CFAEB9400FBC3E813C313F8EA28FA47
:100A1D00EB3400FB8A408B41C3EB94024002C2666B
:100A2D007802EBC4FE7B00EAC4540F4EFAC3EA9879
:100A3D00FA4005C3940250027A027892E6FF3060C4
:100A4D0002414B855192855293D26043E680C3E4B7
:100A5D009AF8E49BF930660241D7E8FAE9FBD3E94D
:100A6D0013FDE813FC88518952C3EF94036038EFEE
:100A7D0020E00DE82CF8E93DF9ECFAEDFB020AA0B7
:100A8D00E828F8E939F9C3E82402F8E93400F97ADD
:100A9D00FE7BFFC3EF9403400E8A538B54884D8920
:100AAD004E8C4F8D50610B885389548A4D8B4E8CD3
:100ABD004F8D503069127553F07554FF754FF075A9
:100ACD0050FF7551F07552FF610BE8FAD3E813FC36
:100ADD008851C3EF94036020EF20E007E82CF8EC79
:100AED00FA41F7E8282402F87AFEC3EF9403400890
:100AFD008A53884D8C4F610B88538A4D8C4FE56816
:100B0D00C3335002646BF5683060026115753402B1
:100B1D00D26043E680E52D54066034A840A941C358
:100B2D00E913F9E813F8C3E913F9E813F830690488
:100B3D00E92440F9C2AF53E67F759100C3E498F5FF
:100B4D0094E499F595759104D26043E680D2AF2275
:100B5D00D264754300752000306C03752040020B84
:100B6D007CD264754300752040306C03752000788D
:100B7D00017901206620E52D54066002C2647914C6
:100B8D00E541C313700104F8C39414400278143086
:100B9D006904781B791B206010E543600C306903F4
:100BAD00D53404D26D8126711D0543E59B5440B5A6
:100BBD002002811030690908C3E89940011861A32A
:100BCD0020640A08C3E8994002617C61A3C264C233
:100BDD00AF53E67F7591003066127594007595F8E8
:100BED00759104D26043E680D2AF617CE5417EFF12
:100BFD00C3334005C3334001FEC3E49E759400F535
:100C0D009561EDC3E53394015002617C306402615E
:100C1D007CD802812461A3C26DC2AF53E67F75916A
:100C2D0000855394855495759104854D92854E9309
:100C3D00D26043E680D2AFE52D54066008206A02EB
:100C4D000533020C62306D0D206C0A20640715818E
:100C5D00158102153A2278003064027801E5377566
:0F0C6D00F007A4F9E5F028F5F0E9A2F013A2F1E1
:100C7C0013A2F213F537C394785003753778C3E594
:100C8C003795384008D265C295C293C2973060023E
:100C9C008199854F92855093D26043E68022D28110
:100CAC00207D16C2AF754202C296D294306202D237
:100CBC0093D2AF759F11020EA6C2AF754202C296B7
:100CCC00D292306202D295D2AF759F11020EA6C29B
:100CDC0081307243207D20C2AF754203900138757C
:100CEC007B40C293C292306204D29781FBD296D2DF
:100CFC00AF759F13020EA6C2AF75420390013875F3
:100D0C007B40C295C294306204D297A11BD296D27A
:100D1C00AF759F10020EA6207D17C2AF75420390CF
:100D2C000113C293306202D297D2AF759F13020E99
:100D3C00A6C2AF754203900113C295306202D297DE
:100D4C00D2AF759F10020EA6D281207D16C2AF7550
:100D5C004204C294D292306202D297D2AF759F10E5
:100D6C00020EA6C2AF754204C292D294306202D275
:100D7C0097D2AF759F13020EA6C281307243207DAD
:100D8C0020C2AF754205900127757B10C297C296A1
:100D9C00306204D295A1A5D294D2AF759F11020EE8
:100DAC00A6C2AF754205900149757B04C297C296E5
:100DBC00306204D293A1C5D292D2AF759F11020EAC
:100DCC00A6207D17C2AF754205900109C29730620B
:100DDC0002D295D2AF759F11020EA6C2AF75420515
:100DEC0090011DC2973062EBD293D2AF759F110266
:100DFC000EA6D281207D16C2AF754206C292D29643
:100E0C00306202D295D2AF759F13020EA6C2AF7597
:100E1C004206C294D296306202D293D2AF759F1022
:100E2C00020EA6C281307244207D20C2AF754201F1
:100E3C00900149757B04C295C294306204D293C16F
:100E4C004FD292D2AF759F10020EA6C2AF7542015F
:100E5C00900127757B10C293C292306205D2950225
:100E6C000E70D294D2AF759F13020EA6207D17C2BE
:100E7C00AF75420190011DC295306202D293D2AF80
:100E8C00759F10020EA6C2AF754201900109C29364
:100E9C00306202D295D2AF759F13C26522900107C2
:100EAC00757B00C295C293C297C294C292C296C27D
:100EBC006222788076FF0876FF0876FF0876FF08B6
:100ECC007603087604087608087603087601087617
:100EDC0001788C76010876FF0876FF0876FF087695
:100EEC00FF0876FF0876030876FF0876FF0876FF82
:100EFC000876250876D00876FA0876FA087604087B
:100F0C0076FF08760108760008767A0876FF087670
:100F1C0001087601087600087603087600227887A7
:100F2C00E6FFC272BF0302D2727888E6C3940360F4
:100F3C0008C27DE630E102D27DC27E7889E630E1DE
:100F4C0002D27EC3EF94026008758E01D273020F39
:100F5C0062758E00C273227880E6149000809378BC
:100F6C00A5F67881E6149000809378A6F67886E64C
:100F7C001490008D9378A7F67886E6F539C3940221
:100F8C005003753902789CE67538FFB40203753846
:100F9C00A0B4030375388278A3E61490009A93F5F5
:100FAC0066D1A922227896E6FA7897E6FB7888E64D
:100FBC00B40305C3EB940EFB307F047A007BFFC3B4
:100FCC00EB9AFCC3948250027C827572000572EC21
:100FDC008572F0A4C3E5F0947D40F222D27FF1B18A
:100FEC001205A01205A07A007B007C10120596E574
:100FFC005C2AFA74003BFBDCF37C04C3EB13FBEAC6
:10100C0013FADCF7FEC27F120FB122757C00757DDE
:10101C0000E5EF20E6037520000520903FFFE5205A
:10102C00146006901DFF1460009304600375EF16A6
:10103C0053D9BF7581C043FF8012059175EF0643EC
:10104C00B203E5B3240220E70DF521E5E320E00629
:10105C008521B343E301120EA97580FF75A40275B7
:0E106C00F1B275D4DF75900175A5FC75F2FE2A
:10107A0075D50175A60175E241120EA9E4F8F6D8F4
:10108A00FD756801120EBE12158B7898867375303D
:10109A0001C2AF1205AA1205BA1205A01205C112A1
:1010AA0005A01205C81205A01216B41205AA120547
:1010BA00AA1205A5C2AF757C00757D0078FA79FA87
:1010CA00308507D9FBD8F7021C00120F2A120F63CA
:1010DA00120FB0120FB178988673120EA975881084
:1010EA0075890275C82475910475D84075A822754A
:1010FA00B80275E690759B80759D0075D10E75BC1A
:10110A005875BB0875BA1175E880120591D2AF12ED
:10111A00084975360053DACF207E0343DA20307E41
:10112A000343DA1043DA01C2D8C2711205AAD261A6
:10113A007B037A0CE55B70077A0CDB030210BE12A4
:10114A0005A02070030210BEC270E55CC394024081
:10115A00E1E52F541F855E5DF55EB55DD5DAD5C232
:10116A006153DACF207E0343DA20307E0343DA105C
:10117A00C2D8C27178A2E67008D274E52F54E0F59D
:10118A002FC2757529001205A5307409C3E5299483
:10119A000A4002D27512059678023074027800C3AA
:1011AA00E55C9840F0C2AF1205BA1205BA1205BA48
:1011BA00D2AF1205AA754C007888E6B4030241BE84
:1011CA00120596788CE6C3940150030212BEE530EC
:1011DA00C3940150030212BE757CA5757DF120747B
:1011EA0035C3E55C94FF50030212BEC2AF1205CFAD
:1011FA00D2AF1205A5C3E55C940150EFC2AF120548
:10120A00BA12059B1205BAD2AF1205A5C3E55C94C2
:10121A00FF40E90217397F05D27F120FB11205A5E7
:10122A00C2AFC27F120FB1AE5CC3E55C947FD2AF8E
:10123A00500241CE120591C2AF1205CFD2AFDFD80C
:10124A00120FE8C3EE94057897F61205AA1216BC97
:10125A007F0AD27F120FB11205A5C2AFC27F120F49
:10126A00B1AE5CC3E55C947FD2AF50E4120591C283
:10127A00AF1205BA12059B1205BAD2AFDFD4120F0C
:10128A00E8EE24037896F6F87997E7C39482400348
:10129A00985006E824827897F61205AA1215D912F0
:1012AA0016EB1205A5120FB1C3E55C94FF5002219B
:1012BA00E2021739757C00757D00C3E55C954C40E8
:1012CA0003855C4C1205A578017988E7B403027896
:1012DA0005C3E55C98400221C2C2AF1205CF1205D0
:1012EA00CF1205CFD2AF1205AA753000E4F531F559
:1012FA00320531E531F4703F0532789AE6781914EF
:10130A006012783214600D787D14600878FA1460DF
:10131A0003753200C3E53298401D120EA9120591D9
:10132A00153275310078998673C2AF1205CFD2AFE4
:10133A00789886731205A512059BE52A7005307404
:10134A000201BE78012074027806C3E55C9840A1C8
:10135A007888E6C3940360031205A5E52A700302A0
:10136A0010BEC2AF120EA9E4F522F523F524F52525
:10137A00F526F567D2AF7885E6C333F565E4F5441B
:10138A00F545F546F547F548F570F52CF52DF53791
:10139A0075700875BB1012059112084D30EDFDA845
:1013AA00BDA9BEE97001F8887112085175700875F7
:1013BA00BB10120F2AC2AF7561FF1208C7852261DE
:1013CA00852262852263D2AF7522017524017525B3
:1013DA0001752601856069756A017888E6B4030794
:1013EA00C27D307602D27DD268D269753300120D81
:1013FA00FE120E2F1208E71208EE1208E71208EE84
:10140A001208E7120B6E1206B0120C63120CAA1223
:10141A0008EE120B5D306E031206B1206603120845
:10142A0003306603120833120C63120CDB1208EE47
:10143A00120B6E306E031206ED120C63120D54126B
:10144A0008EE120B5D306E0312074B120C63120D7D
:10145A00851208EE120B6E306E031207A8120C6387
:0F146A00120DFE1208EE12084D120B5D120C63EC
:10147900120E2F1208511208EE30692F856461850A
:101489006462856069756A0179187A0CC3E53399D4
:10149900400CC269D26A8A357561FF0214B4C3E58A
:1014A9005C9401400302140D021542306A25206C38
:1014B90022E535147006C26AD26B810DF535C3E594
:1014C9005C9401400302140D7888E6C39403600319
:1014D900021542753600788279A4E760027803C361
:1014E900E55F985054307404E52A604D7888E6B475
:1014F9000317207D05207607A112307602A112205C
:101509006C07D26C856461814C78F0306C05856418
:10151900617820C3E541985002810D306C1BC26C83
:10152900C27D307602D27DD26A75351285646181B9
:101539000D0536E55C6002A145753600C2AF120E95
:10154900A97887E6FE7602120F2A7887EEF6E4F587
:1015590022F523F524F525F526F565752C00752D5D
:1015690000D2AF1205A5120EA978A4E66006D2959D
:10157900D297D293307409C3E5369404400201BE70
:1015890041F6901A0D782012161BE520B45A0CA3C7
:1015990012161BE520B4A5030215B9757CA5757D46
:1015A900F1120EBE1215D9757C00757D000215D891
:1015B900901A0378807B0A12161BA308DBF9901A8C
:1015C9000F788C7B1912161BA308DBF9901A2822B5
:1015D900C2AF12165E12163B901A00740E12162034
:1015E900A37409121620A37415121620901A0378F1
:1015F900807B0A12161FA308DBF9901A0F788C7BDF
:101609001912161FA308DBF912167112164F901A38
:101619002822E493F622E6438F01538FFDFFC3E5A9
:1016290083941C400122EF857CB7857DB7F0538FE9
:10163900FE22438F02438F01857CB7857DB7901ABF
:101649000DF0538FFC22901A0D745AD120901A0E66
:1016590074A5D120227A3079D07820901A40D11BF4
:10166900E520F709A3DAF7227A3079D0901A40E712
:10167900D12009A3DAF922AB74A875BB01027984D8
:10168900BB02027985BB03027986BB04027992BB4E
:1016990005027987BB060279A3BB0702799CBB08BF
:1016A900027988BB09027989E8F7227C051205AA23
:1016B900DCFB22C2AF1205BA1205C11205C8120518
:1016C900CF12059B1205BA1205C11205C81205CF22
:1016D90012059B1205BA1205C11205C81205CFD20F
:1016E900AF22C2AF1205CF1205C81205C11205BA41
:1016F90012059B1205CF1205C81205C11205BA12AF
:10170900059B1205CF1205C81205C11205BAD2AF41
:1017190022AE74AF75C2AF1205BA1205BA1205BA74
:1017290012059BDEF21205CF12059BDFF8D2AF221C
:10173900D1BCD1B4D1B4757401757501757600F158
:101749001A7C05AD5C1205AAC3ED955C70F5C3E57D
:101759005C9401400AC3E55C94FF4032021775D1DD
:1017690080B1D9D1BCC2AF75EF16D1B4DCD505763D
:10177900C3E5769403500280C6D1B40575E57414A7
:1017890090009F93F808C3E57598500280AED1B4D4
:10179900D1B40574C3E574940A5002809C120EBE3C
:0917A900B1D9C2AF75EF16D1B43D
:0319FD00021017BE
:101A00000E0915FFFFFFFF0304080301015AA5019A
:101A1000FFFFFFFFFF03FFFFFF25D0FAFA04FF01DE
:091A2000007AFF0101000300FF40
:101A400023534B4D6F6E73746572383041232020E1
:101A500023424C48454C4923463333302320202031
:101A60002020202020202020202020202020202076
:101C0000C2AFC2D353D9BF7581C043B20343FF8073
:101C1000752438752503B1DC7529A5752AF175E29F
:101C20004043F12053A4DF75D4FFD2857DFA7803B9
:101C300079E67C10752200752300901DE97B0675FE
:101C400024987525013085028145208508D8FBD967
:101C5000F9DCF781B7308508D8FBD9F9DCF781B713
:101C6000B19CE493A3C39A6004DDC381B7DBDBB10D
:101C70008E6002812E7B08E493FAA3B16FDBF87AC1
:101C800030B16F752200752300B18EEAFCEBFDC305
:101C9000ED94FE400EB18E8A278B28ED30E0048A49
:101CA000828B83B18E7AC270D8C3ED94FE601950D6
:101CB000CEBD002BEC600F7520007521FF7529004B
:101CC000752A000200008100A827A9280809D80465
:101CD000D90281DCB192EA89AAF281CE0D81A3C337
:101CE000ED94035053EDA2E092007AC5C3E58294CF
:101CF00000E583941C508A200010438F02438F011B
:101D00008529B7852AB7F0300029A827A92808090E
:101D1000438F01538FFDD804D902A133C3E58394C7
:101D20001C4003A3A11689AAE28529B7852AB7F02A
:101D3000A3A116538FFC817F7AC1BD030CE493A34A
:101D4000FAB153DCF8B14B817F8181AA22AB23B178
:101D50006FEBFAEA6222752608C3E52313F523E543
:101D60002213F52250066323A0632201D526EAB18F
:101D7000DCB1DC75260AEAF4200102D285300102CA
:101D8000C285B1DCC3134002C201D526EB22B19259
:101D9000EAFB208502A192308502A197752608AE44
:101DA00024AF25C3EF13FFEE13FEB1E0B1DCC3EAAD
:101DB000133085024480FA30E703632201C3E52330
:101DC00013F523E52213F52250066323A0632201B5
:101DD000D526D9E52265236523F52222AE24AF2539
:101DE0000E0FDEFEDFFCD20122424C48656C6934E6
:071DF000373164F3300601F6
:00000001FF
